:020000040000FA
:020000000528D1
:0800080029298312031385016D
:10001000831606309F00CF30850007309C00831682
:100020000030850086000F308700FF3088001730D1
:1000300089008C178312C0308B00C00185018601B6
:100040008701880189010221B220E1209620E12068
:10005000A120AC20C720E4203808F620D42037089F
:10006000F620D4203608F620D4203508F620D420F7
:100070003408F620D4202E30D4203308F620D420A3
:100080003208F620D4203108F620D4202030D420A5
:100090003A08F620D4203908F620D420AF20E420F6
:1000A0002030D4203008F620D4202E30D4203F0831
:1000B000F620D4204B30D4206830D4207A30D4209D
:1000C0002030D4202030D4203E08F620D4202E30FA
:1000D000D4203D08F620D4203C08F620D4204B3014
:1000E000D4206830D4207A30D4202928820746349E
:1000F000723465347134753465346E3463347934F4
:1001000020344334683461346E340034820742341E
:1001100061346E34643477346934643474346834EC
:10012000203420344234463430340034C001AC2012
:1001300040087620003A0319A028D420C00A972846
:100140000034C001AF2040088620003A0319AB28D4
:10015000D420C00AA22800340030C5000034013089
:10016000C5000034AC202030C7202830C72006301E
:10017000C7200C30C720F320AF202030C720283004
:10018000C7200630C7200C30C720F3200034C4003D
:10019000440E0F3986008510192144080F39860056
:1001A0008510192108210034C400440E0F3986003F
:1001B0008514192144080F398600851419210C2152
:1001C00000348030C7200034C030C7200034803E67
:1001D000C7200034C03EC72000340D30C720003493
:1001E0000C30C72000340130C72000340F39C6005E
:1001F000093C031CFC28FF284608373E0800460837
:10020000303E080064300D2932300D2914300D299C
:100210000A300D2905300D290130C100C730C20058
:100220000130C300C20B1529C30B1229C10B0E29C3
:100230000034451C1F21451C0034242100340515C1
:100240000000051100000034851500008511000034
:100250000034A200030E8301A00007080F39303ECE
:100260008400080880008C13200E8300A20E220E4A
:02027000090083
:02400E00723FFF
:00000001FF
